:1000000003C003C003C003C003C003C003C003C0D8
:10008000A5C3CFC3CEC3CDC3CCC3CBC3CAC3C9C31F
:10009000C8C3C7C3C6C3C5C3C4C3C3C3C2C317C0D1
:1000A00016C04CC014C009021200010100803209C0
:1000B000040000000000000012011001FF00000811
:1000C000D01653070B01000000010403090411249A
:1000D0001FBECFE5D2E0CDBFDEBF00EB0F9307E040
:1000E0000F9310E0A0E6B0E0E8EEFFE102C005905B
:1000F0000D92A636B107D9F720E0A6E6B0E001C020
:100100001D92A639B207E1F7E2C1A82FB92F80E00E
:1001100090E041E050EA609530E009C02D918227DF
:100120009795879510F084279527305EC8F36F5F09
:10013000A8F30895EADF8D939D930895CF93CFB7E9
:10014000CF93C0915F02C03B21F4C0915E02C730E3
:1001500021F0CF91CFBFCF91A1CFCC27C395B39B37
:10016000E9F7B39B0BC0B39B09C0B39B07C0B39B1C
:1001700005C0B39B03C0B39B01C0D3C00F92DF93F4
:10018000C0917900DD27C058DF4F012EB39B03C01B
:10019000DF910F90E6CF2F930F931F934F932FEF85
:1001A0004F6F06B303FB20F95F933F9350E03BE0B2
:1001B00065C016B30126502953FDC89556B30127D3
:1001C00003FB25F92F7306B3B1F05027102713FB5B
:1001D00026F906B22230F0F000C016B3012703FB67
:1001E00027F90126502906B22430E8F54F77206818
:1001F00016B30000F6CF50274F7D206206B2102FB5
:10020000000000C006B300265029102713FB26F972
:1002100006B2E2CF4F7B06B3206400C0DACF0126DE
:100220005029187106B269F14E7F2160012F16B373
:1002300028C0002650294D7F06B22260102F29C009
:10024000012650294B7F06B22460012F2DC016B322
:1002500001265029477F2860000006B22EC04F7E3D
:1002600006B3206130C0422706B3499300265029C7
:10027000102706B24FEF13FB20F9297F16B379F24E
:10028000187159F10126502906B2012703FB21F903
:10029000237F06B371F2002650293150D0F006B208
:1002A000102713FB22F9277E16B351F2012650299D
:1002B000012703FB06B223F92F7C49F2000006B3A5
:1002C000102713FB24F90026502906B22F7939F2A2
:1002D00070CF10E21ABF002717C03B503195C31BE7
:1002E000D04010E21ABF0881033CF9F00B34E9F06A
:1002F000209177001981110F1213EDCF093651F1BA
:100300000D3211F0013E39F700937E003F915F916D
:100310004F911F910F912F91DF910F90CAB7C5FD9B
:100320001DCFCF91CFBFCF91189520917E00222372
:1003300069F310917C00112321F5343022F13093C0
:100340007C0020937800109179003BE0311B3093C2
:10035000790019C000917C0001309CF40AE53091CD
:10036000600034FD11C000936000CCE6D0E010C006
:10037000052710E000C021C0052710E0C89508BB84
:1003800014C03AE501C032ED032EC0E0D0E032E007
:1003900017B31861C39A08B317BB58E120E84FEFB1
:1003A00020FF052708BB279517951C3F28F700005D
:1003B0004552B0F720FF0527279508BB17951C3F2E
:1003C000B8F629913A9561F7077E10917D00110FDB
:1003D00008BBC250D04011F01093770010E21ABF52
:1003E000086017B3177E402F477E54E05A95F1F707
:1003F00008BB17BB48BB8ACFF8942FEFB0E8A0E446
:100400004AE0B1BF000081EE9CE0B399FECFB39B00
:10041000FECF0197B399FDCF97FF03C0BA1B81951B
:1004200001C0BA0FA69529F4281710F031B7282F6C
:10043000A1E0415031F731BF000078940895F8945D
:10044000F201329785E080935700E89578940895FB
:10045000F201309729F4909368008093670007C0F9
:10046000E430F10539F490936A00809369008FE5D8
:100470009CEC1FC02CEB421628E1520639F4809107
:100480006700909168008E559C4F13C02EEB42166A
:1004900028E1520639F48091690090916A008D55E7
:1004A0009C4F07C02AEB421628E1520611F481B78F
:1004B00090E02FB7F89431E00C0130935700E895A5
:1004C00011242F0182E0480E511C2FBF089504B65D
:1004D00001FC14C0EDEBF8E1E491EF3F79F0F89402
:1004E000BB9A1BBE15BA10925F02EAEBF8E1E491E9
:1004F0008E2F81508E3F08F462C163C114BE88E123
:1005000081BD87E081BDBB9A88E893E1ECE9F1E029
:100510003197F1F70197D1F7BB98AC9A8BB780620E
:100520008BBF7894712C8CE991E00197F1F7A89535
:10053000312C60917C00162F135017FDB2C08091B2
:100540007900CCE0D0E0C81BD109C058DF4F615022
:10055000CE01DBDD8E3F9F4409F0A1C08091780081
:100560008D3209F085C0183009F099C083EC809372
:100570006C008AE580936000109266009881292FB4
:10058000207689812223D1F0712C811108C082E666
:1005900090E090937B0080937A0024E05FC08130EC
:1005A00051F481E180935700E8954C805D8097FD80
:1005B00050C02FEF4FC0382E20E050C09A811092CB
:1005C0007500811106C01092760085E790E022E068
:1005D0003BC0853019F490937D002CC0863009F51E
:1005E0008B81813019F48AED98E104C0823041F4A6
:1005F00088EC98E190937B0080937A0022E10DC013
:10060000833051F4911108C08CEE98E190937B00F7
:1006100080937A0024E001C020E080E480936600AB
:100620001DC0883059F0893019F490937F0002C0C2
:100630008A3039F085E790E020E006C08FE790E04F
:1006400002C085E790E021E090937B0080937A00E0
:1006500005C02E8180E88093660007C08F818111DC
:1006600004C08E81821708F4282F2093610017C0E0
:100670008091660087FF13C080EC481688E1580619
:1006800020F0842D8F7339F00AC089919991E0DEB2
:10069000125091F7F6CF95E0392E1092610010922A
:1006A0007C008091600084FF42C0809161008F3F98
:1006B00009F43DC0182F893008F018E0811B8093A1
:1006C000610080916C0098E8892780936C00112369
:1006D00011F1E0917A00F0917B008091660086FF35
:1006E0000BC0ADE6B0E084918D9331968DE690E03D
:1006F000810F8A13F8CF0BC0EF01ADE6B0E089910E
:100700008D93FE018DE690E0810F8A13F8CFF09370
:100710007B00E0937A00612F8DE690E00BDD1C5F9B
:100720001C3019F08FEF809361001093600084E11A
:1007300096B3987131F48150D9F710927D001092E0
:100740007700C1E08111C0E080916B008C1729F027
:10075000C11101C051DEC0936B00C30101963C0181
:100760008035934C11F484E0382E232D3320E9F0AA
:100770008AE390E20197F1F72230A9F4F894E0ECD3
:10078000F8E1E054F10983E080935700E895309751
:10079000C1F7412C512CC8E08FEF9FEF59DEC150BB
:1007A000D9F74DDE02C02530E1F384E03812BBCE2C
:1007B000EDEBF8E1E491EF3F09F4B5CE90CEE1BF67
:1007C00000006BCCFFCF5AFF18BA400800000000B1
:1007D0000000000000000000000000000000000019
:1007E00000000000000000000000000011241FBEF7
:1007F000CFE5D2E0DEBFCDBF10E0A0E6B0E0E8E894
:10080000FAE002C005900D92A236B107D9F710E0C8
:10081000A2E6B0E001C01D92A236B107E1F71CD1FB
:1008200031C12ECC05C0EDE1F0E13197F1F7019730
:100830000097C9F70895AC01407C80E090E0FC018E
:10084000E40FF51F25913491FC01EE7FE60FF71FB1
:100850002083318302968034910589F70895FC0145
:10086000E07C83E080935700E89507B600FCFDCF5D
:100870000895CF93DF93EC01AB01DB0120E030E082
:10088000FE01E41BF50BEA0FFB1F8D919D9161E0CA
:100890000C0160935700E89511242F5F3F4F2032E1
:1008A000310571F785E0FE0180935700E89507B6A2
:1008B00000FCFDCFDF91CF910895CF93DF93CDB7AB
:1008C000DEB7C054D0400FB6F894DEBF0FBECDBF28
:1008D0008091600090916100969587958150904439
:1008E000FE0131969E012F5B3F4F81939193E2175A
:1008F000F307D9F780E090E0B2DF80E090E0BE013E
:100900006F5F7F4FB6DFC05CDF4F0FB6F894DEBF7E
:100910000FBECDBFDF91CF9108950F931F93CF935B
:10092000DF93CDB7DEB7C054D0400FB6F894DEBF2A
:100930000FBECDBF00E010E040C080E090E0F801C5
:10094000E256FF4FE80FF91F9C013595279547E0C8
:10095000EC3CF40770F0F901EE0FFF1F21E030E0EE
:100960002C0F3D1FE20FF31F2FEF3FEF318320834A
:100970000DC045915491F901EE0FFF1F21E030E0C9
:100980002C0F3D1FE20FF31F4083518302968034EA
:100990009105A9F68091600090916100800F911FF0
:1009A0005EDF8091600090916100800F911FBE0119
:1009B0006F5F7F4F5EDF005C1F4F37E0003413072F
:1009C00009F0BBCFC05CDF4F0FB6F894DEBF0FBE9F
:1009D000CDBFDF91CF911F910F910895CF93DF93FA
:1009E000CDB7DEB7C054D0400FB6F894DEBF0FBE0F
:1009F000CDBF80E090E0BE016F5F7F4F1CDF8FEFC7
:100A00009FEF9A83898380E090E029DF80E090E087
:100A1000BE016F5F7F4F2DDFC05CDF4F0FB6F894D4
:100A2000DEBF0FBECDBFDF91CF910895CF9387B3C7
:100A3000836087BBC198CAEF81E090E0F3DEC19A82
:100A400081E090E0EFDEC198C150B1F7CF910895F9
:100A5000E0E0F0E00995089588B318BA87B38FEF06
:100A600087BB8AEF90E0DEDE87B317BA8AEF90E0AB
:100A7000D9DEF894B3DF51DF20DFD8DFE9DF80E093
:080A800090E00895F894FFCF07
:020A8800C01894
:040000030000008079
:00000001FF
